:020000000429D1
:0800080003299000F8309E006E
:1000100000009E0B08281008080090000A309F007E
:1000200005209F0B10281008080090006430A000E5
:100030000520A00B18281008080090006430A100CB
:100040000D20A10B202810080800F3308D000000BF
:100050008D0B27280800FF309500010893008515B7
:100060008511950A0108130603192F281508FF3C6E
:1000700094000800031020309D009C019B019A0110
:100080009901940D930D920D910D9C0D9B0D9A0D60
:10009000990D9D0B4C2808001C30840059201B3002
:1000A000840059201A3084005920193084005920C6
:1000B0004128033000078C008C1980003030000785
:1000C0008C008C1B8000080022148230EE20190E58
:1000D0000F398B2019080F398B202030D9201A0EA8
:1000E0000F398B201A080F398B201B0E0F398B20EC
:1000F0002030D9201B080F398B201C0E0F398B2084
:100100001C080F398B202030D9204830D9207A3074
:10011000D92022100800003A0319902822109528AF
:10012000221C95282030D9200800F63E0318073EEF
:100130003A3ED920080005100000851000000D206F
:100140000F3086053030860483160F300605860092
:1001500083120514000005100D2005140000051081
:100160000D2005140000051015200F3086052030E5
:1001700086040514000005102830C3200830C32071
:100180000C30C32006308F0015200F3086050F0875
:10019000F0398604000085100000051400000510E9
:1001A0000F3086050F0EF039860405140000051087
:1001B000080005208514960006080F3986001608E9
:1001C000F039860405140510960E06080F398600CE
:1001D0001608F03986040514051000340520851032
:1001E000960006080F3986001608F03986040514B3
:1001F0000510960E06080F3986001608F039860499
:10020000051405100034090085018601831610309D
:1002100085000F3086002730810000308B0083126C
:1002200005159B200C30EE202830EE20E2308E00A9
:100230000130EE2005202030D9204630D920523020
:10024000D9204530D9205130D9203330D92032300F
:10025000D9202D30D9204C30D9204C30D9202D3008
:10026000D9203230D9203030D9203130D920323025
:10027000D9202030D9201D201D201D200130EE2046
:10028000052015202030D9202030D9203130D92028
:100290003630D9204630D9203830D9203430D920D2
:1002A0002030D9205130D9203D30D9203430D920C8
:1002B0004D30D9204830D9207A30D9202030D9206B
:1002C0002030D9202030D9201D201D201D200130B4
:1002D000EE200520152003309700E73098008101BB
:1002E00092019101831685158312252000000000DC
:1002F00000000000000000000000000000000000FE
:1003000000000000970803198829000000008B29CD
:1003100098080319A32925209803FF301806031D08
:10032000922997030B1D9D290B11920A03199B29F2
:10033000000000008229910A8229000000000000CC
:100340000000000082298316851183122B203A2099
:100350006420990803199A0803199B0803199C083B
:100360000319B4298E016B298E0A0319B8296B2948
:100370000130EE2005202030D9204130D9205230E4
:10038000D9205230D9204530D9205430D9202030BE
:10039000D9204130D9205530D9205430D9204F3080
:1003A000D9202030D9202030D9201D201D201D200B
:0803B0001D201D200511DB29B1
:02400E00F13F80
:104200004634723465347134333432345F344C3470
:104210004C345F343234303431343234203420344E
:1042200050344934433431343634463438343434F9
:10423000203451343D3434344D3468347A342034AD
:02424000003448
:00000001FF
